:20000000C5402703BDFE63BDF03CD663C5202703BDF06E8D0220AF96282A08B7700001A62B
:20002000002B023131395FF77F0CD727962580172C028B18B77F0D97267EF34F5FF77F0C55
:20004000D727D7817EF34F9627814F270F7F00814CB77F0C9727DE2308DF2339D6282B0A04
:20006000D663C51027047C0081398DD0200096269125270A8117260286FF4C7EF0347D0041
:200080005226367D002827037EF02ED665C50826F74C81182D014F9725B77F06BDF0349057
:2000A00027C200D7D897D9DED8C6504FB7700001A700085A26F6DE2339BDF3B596258017DF
:2000C0002A028B1820B59627270C4AB77F0C9727DE2309DF2339864FB77F0C972720009672
:2000E00026260286184AB77F0D97269125260F7D0052270ABDF3B59625B77F0D97267EF34E
:200100004F7D0028275BBDF1F29627DE23DFD820049CDC2726814F272A084C9CD8271CB788
:20012000700001E6002AEA814F271F084CB7700001E6002A069CD8271E20ECB77F0C9727E7
:20014000DF2339BDF06A962720D1BDF06A962720DC9627DFD820D0BDF026BDF0C64FA7002F
:20016000397D002F272D2B2C4FD6279B2F814F2205112E0520F57EF06A36D6239624902711
:20018000C20030AB00C900D723972432B77F0C9727DE23399627814F27127C0027BDF2922E
:2001A000E50027F09627B77F0C7EF34F7EF06A7D0028277A8D3C9627DE23DFD88D1F2B133E
:2001C0009CD827169CDC27128D132AF4DF2397277EF047BDF1DD2BFB20E67EF13B4D2709AC
:2001E0004A09B7700001E60039DF23BDF0D6962720F0962597DD4FD652271DC404F87802EF
:20020000C5042714860898218B0797DAC6D4D7DBDEDAA60097DD8608982197DC96DD8017AE
:200220002C028B18BDF341DBDCD7DC97DD397D002F27242B14D6272605BDF0C6D6274F9B2D
:200240002F112BFB902F7EF179BDF0C696272707BDF292E50027F239CE0030C60A4FA700F7
:20026000085A26FA20218D2AEA00E700D62FCA80201D8D1E53E400E700CE0030C60A4FA120
:2002800000260E085A26F8D62FC1D02704C47FD72F39CE00309627444444BDEE9CC601963C
:2002A0002784072704584A26FC39BDF9C0847F80202B0A81502D042E0486D0972F39BDF9D7
:2002C000C0D664C54026014A81302C02863081312F0286318401D652260F4848F67802C4D9
:2002E0000411271DBDF388201836C404B678028404112606335D27092004335D2603BDF3F5
:2003000088BDF9C08D3381182D0286179B254C81182D028018B77F0D9726BDF9C08D1A81B0
:20032000502D02864FB77F0C9727BDF34F96638502270DBDF0177EF151847F80202C014F13
:20034000391648481B5F48594859485948593996268DEE9B27D921D7239724DE23398130F4
:200360002B1481392F0C84DF81412B0A81462E068007840F0C394F0D3944444444840F81DC
:200380000A2D028B078B30397D0015263B966085202635C6078D20B7700001A60095282789
:2003A000279652270D8404F67802C4041127037EEFE37EF151C606D782BDF3C9B678028899
:2003C00004B778028D16DE233996218B07977D86D0977ECE0021DF7FC6302036CE0021DFDC
:2003E0007DB678028404488B8097218B07977F86D097807D00522704D6822002C6308D129F
:200400009625B77F069626B77F0D9627B77F0C7EF34FDE7FB7700001A60008DF7FDE7DB784
:20042000700001A70008DF7D5A26E7390000000000000000000000000000000000000000A0
:2004400000000000000000000000000000000000000000000000000000000000000000009C
:2004600086022027860320238604201F8605201B860620179664852026698607200D860819
:20048000200986092005860A2001439789BDEEAB7F007A4FCE0004BDF990CE0000BDF99B96
:2004A000CE00027EF99BBDF79A96892A05CEF528200FD665C420D791CEF4E448BDEE9CEEFA
:2004C00000AD009689810A270E9656270ABDF7B296572703BDF7B2BDF5E1CE0007BDF992E0
:2004E0007EF99939F4E3F4E3F557F557F55FF55FF6C5F6C5F513F4FAF534B67802D65227B1
:20050000029852840444448A30D664C54026014CBDF7B296264A90252C028B188B20BDF722
:20052000B296278B207EF7B2B6005BBDF7B29689437EF7B2CE7B80DFD8A61E810D2617A6C5
:200540001F818A2611847F9789DED8A60008DFD8BDF7B24D2AF339BDF5D8BDF03C2017BD8C
:20056000F5D89652270DF678028404C404112703BDF3B5BDF0264FB7002E978ABDEE7A7D68
:20058000007A2B2DBDF609D6602A0481032722C5102706DE239C8527184D2703BDF7B2DE7E
:2005A000239C85270CBDF5FE7D002726CF8D0320CB3996658510270496282B1B96582717DC
:2005C000BDF7B2965927107EF7B23696912607965A2703BDF7B23239DE26DF87DE23DF8524
:2005E0003996282615968981022D0F81062E0B2D06D664C5202703BDEFF17F008939BDF024
:20060000477D0081271E7EF06ADE23B7700001A6007D0028260F16C4F0C190260286208462
:200620007F7F009139D689C501264BD68A4D2B0BC10126F07F008A8D9120E481E02726C107
:200640000227DCC601D78A9C852729847F91DB2608D689C406C106271CBDF5FED62726A9B0
:20066000BDF5B220A4C10227DAC1012603BDF5CAC60220D14F394D2B167D008A27A13696BD
:2006800055BDF7B28628BDF7B27F008A32209016C4F0C1902617369655BDF7B28647BDF740
:2006A000B232840FBDF37DBDF7B27EF6597D008A2610369655BDF7B28629BDF7B28601976C
:2006C0008A327EF61FBDF5D85FD7DCD7DDD78AF67802C404D7DE96648520270E861C97DA46
:2006E00097DBB7700001A7002023860297DA860397DB965227088404112603BDF3B5962589
:20070000BDF341DB218B4FC900D7DC97DD9652270D8404F67802C404112703BDF3B59625EB
:2007200080172C028B18BDF341DB21D7D897D9F67802C404D1DE2703BDF3B5DE239CD82733
:2007400029BDF0C6B7700001A600847F91DA27069CD826ED2014D664C5202706D626D18739
:200760002605BDF5FE2003BDF06ADEDCDF85BDEE7A7D007A2B20BDF6094D270791DB2717FE
:20078000BDF7B2DE239C85270EBDF5FE7D002726DDBDF5B220D8397EEFE6D690CA01D790C5
:2007A00036F67E00C41C968384831B9783B77A003239367D009026028DE0D68FC10C27FA93
:2007C000DE8D32A70016D80FD70F7C008F088C010C2603CE0100DF8DD683C49FCA20D783E2
:2007E000F77A00397F0090968F27078601BDF9A420F5B67A00850227EE965F260DCEF8320B
:00000001FF
